:020000040000FA
:040000008A114228F7
:08000800FE00030E8301AB00B2
:100010000A08AC008A0139280830AD000310A20D8F
:100020000310A00D031C16282108A207AD0B0E28F3
:1000300008001030AD00A201A3010310A60DA70D0A
:100040000310A00DA10DA20DA30D23082502031D71
:100050002B282208240203192F28031836282508E4
:10006000A3022408A202031CA3032614AD0B1D281F
:1000700008002D08AE002008A8002108A9002208C9
:10008000AA00C329831605108510851205120511D3
:10009000172A0310360CE200350CE1000310E20CC5
:1000A000E10C61083506E30062083606E40003103F
:1000B000360CE600350CE5000310E60CE50C0310E9
:1000C000E60CE50C65086306E70066086406E800D0
:1000D0000310360CEA00350CE9000430A0000310D0
:1000E000EA0CE90CA00B6F2869086706EB006A08A8
:1000F0006806EC0001306B05DF00E0010310360CF0
:10010000E200350CE100E301E4015F18E417630845
:100110006104B50064086204B6003508A000360822
:10012000A1000800492083122008DD002108DE001C
:10013000F430A4000130A5005D08A0005E08A10015
:10014000192083122208DB002308DC0000305C0247
:10015000031DAC284B305B020319B4280318B428E4
:100160004B30DB070318DC0A5B08A0005C08A10029
:1001700008007D147D0883128500FD147D0885002C
:10018000FD167D0885007D167D0885007D157D089E
:1001900085005514D5105511D5155512D512551386
:1001A000D5135610D610922083122008BB002108C8
:1001B000BC00BD01BE01BF01C00192208312200816
:1001C000C1002108C200C301C401CF01D001D10187
:1001D000D201D301121187309205FC309205C33051
:1001E000831692008312C90183168C1483128C101B
:1001F0001215080012117D147D088500FD147D087C
:100200008500FD167D0885007D167D0885007D151D
:100210007D088500080030108C1C132983168C1C67
:100220001329831230148312301C8A298C10490838
:10023000031D45293330C9004F08CA005008CB00C0
:100240005108CC005208CD005308CE004A080319CB
:100250002C297D107D0885004B0803193229FD10DB
:100260007D0885004C0803193829FD127D0885009A
:100270004D0803193E297D127D0885004E0803199B
:1002800046297D117D0885004629C90305304A02AB
:1002900003194C29031C4F290530CA0252297D1429
:1002A0007D08850005304B0203195829031C5B2982
:1002B0000530CB025E29FD147D08850005304C0217
:1002C00003196429031C67290530CC026A29FD162D
:1002D0007D08850005304D0203197029031C732920
:1002E0000530CD0276297D167D08850005304E0249
:1002F00003197C29031C7F290530CE0282297D1534
:100300007D0885004708031D8929CC30C700D61514
:100310008A29C7032808A0002908A1002A08A200EA
:100320002E08AD002C088A002B0E8300FE0E7E0ED8
:100330000900FA305B025C04031DB129D51655177C
:10034000D51756145516BB01BC01BD01BE01BF0136
:10035000C001C101C2015B08C3005C08C4005D1498
:10036000B2295D1020105D1820140800103083168B
:100370009F00953083129F005611991319160C1384
:1003800083160C17080034100C1FCB2983160C1F82
:10039000CB29831234148312341C0B295619E729F4
:1003A0001E08A000FF30A1000C2083122208B0001C
:1003B000B10183161E088312B200B301330831075E
:1003C000B80032083007B7000318B80A56150C13E6
:1003D0000B29561DF2293708B9003808BA00561102
:1003E00020140800201008009F1408008030831299
:1003F0009F0019120800FA20F6218B1383120313B1
:10040000AD30A000E630A1000A128A11A10B042A27
:100410000A128A11A00B022A00000000000000004E
:1004200000000000000000000000630008009F01C1
:1004300083129F019A019C01FA20831203139C30BE
:10044000A0007F30A1000A128A11A10B232A0A12F0
:100450008A11A00B212A0000BA305402031D332A4E
:10046000D630D400362ABA30D400FB2183123508A6
:100470003604031D3F2AE130B500AC30B600B6218A
:10048000B9200B178B178312C801D6118312D61D02
:10049000462AD611E9218312561320185617561FE3
:1004A000652A00303A02031D572AD2303902031957
:1004B000642A031C642A0A304802031D622AC80108
:1004C000FB21652AC80A652AC80183123B083C043F
:1004D00003198D2A3B033C04031D892ABB01BC017F
:1004E000922083122008C5002108C6004508DB00C1
:1004F0004608DC0099218312D7112018D715D71987
:100500008D2AD516D614D5144508BD004608BE0060
:100510008D2ABB033B0A0319BC033D083E040319A3
:10052000B42A3D033E04031DB02ABD01BE01922042
:1005300083122008C5002108C6004508DB004608D4
:10054000DC0099218312D7132018D717D71BB42AA0
:100550005517D61455144508BB004608BC00B42AEC
:10056000BD033D0A0319BE033F0840040319DB2AFB
:100570003F034004031DD72ABF01C001922083120C
:100580002008C5002108C6004508DB004608DC003D
:1005900099218312D8112018D815D819DB2AD5171C
:1005A000D614D5154508C1004608C200DB2ABF0392
:1005B0003F0A0319C003410842040319022B4103F7
:1005C0004204031DFE2AC101C201922083122008A9
:1005D000C5002108C6004508DB004608DC0099215B
:1005E0008312D8132018D817D81B022B5614D614F0
:1005F00055154508BF004608C000022BC103410A3B
:100600000319C203430844040319202B4303440481
:10061000031D1C2BC301C401D6145514D5159220FB
:1006200083122008BB002108BC00922083122008FE
:10063000C1002108C200202BC303430A0319C403CD
:10064000551C2D2BFF304F0203192B2B03182B2B7E
:100650000530CF07362B5510362BD51E362B4F08BD
:100660000319352B0530CF02362BD512D51C432B61
:10067000FF3050020319412B0318412B0530D007DE
:100680004C2BD5104C2B551F4C2B500803194B2BC2
:100690000530D0024C2B5513551D592BFF305102FC
:1006A0000319572B0318572B0530D107622B55110F
:1006B000622BD51F622B51080319612B0530D10223
:1006C000622BD513D51D6F2BFF30520203196D2BF2
:1006D00003186D2B0530D207782BD511782B561CBB
:1006E000782B52080319772B0530D202782B56103D
:1006F000551E852BFF3053020319832B0318832BC0
:100700000530D3078E2B55128E2BD61C8E2B5308FB
:1007100003198D2B0530D3028E2BD610F421462AD7
:02400E00643C10
:00000001FF
